:020000008D2A47
:1000080003088D00820700000000000000000000C7
:1000180000000000000000000000000000000000D8
:1000280000000000000000000000000000000000C8
:100038000800C60A08304602031D2428C601C60A5D
:10004800460882072E283B284828552862286F280A
:100058007C288928FF304602031D3A28C60A033047
:100068004602031D3A28C601013086061D28FF30C6
:100078004602031D4728C60A08304602031D4728C2
:10008800C601023086061D28FF304602031D54288B
:10009800C60A06304602031D5428C60104308606E7
:1000A8001D28FF304602031D6128C60A0B30460290
:1000B800031D6128C601083086061D28FF30460248
:1000C800031D6E28C60A0C304602031D6E28C601A1
:1000D800103086061D28FF304602031D7B28C60AFD
:1000E80004304602031D7B28C601203086061D28E1
:1000F800FF304602031D8828C70A17304702031D30
:100108008828C701403086061D28FF304602031D97
:100118009528C70A09304702031D9528C701803072
:1001280086061D28000000001108062000000000B7
:10013800120806208F0B962808000E34113411344B
:100148000A3404340434043411341B34153411349F
:10015800113411341134113411341134113411346F
:1001680011340E3404340C340434043404340434A8
:100178000E340E34113401340234043408341F347C
:100188000E34113401340634013411340E3402347F
:1001980006340A3412341F34023402341F34103443
:1001A8001E340134013411340E340E341134103439
:1001B8000E34113411340E341F3401340134023436
:1001C8000234043404340E34113411340E3411342E
:1001D80011340E340E34113411340F340134113407
:1001E8000E3400340034083404340234003400344B
:1001F8000234043408340034003400340034003449
:10020800003400340E34113411341F3411341134D5
:1002180011341F34113411341134113411341134A0
:100228000E341E34113411341134113411341E3487
:10023800113411341E34113411341E341034103476
:1002480010341034103410341F34103410341C346B
:10025800103410341F34103410341C34103410345B
:1002680010340134013401340134013411340E34B2
:10027800113410341334113411340E341134113450
:100288001134153413340E34043404340E34113458
:100298001234143418341434123411341B34153411
:1002A8001134113411341134193415341334113410
:1002B800113411340A3404340434043411341B3432
:1002C80015341134113411340A3404340434043428
:1002D80011341B34153411341134113411341934D8
:1002E800153413341134113411340A3404340434F9
:1002F800043407308C00752A04308C00752A7E344B
:1003080030346D34793433345B345F3470347F3453
:10031800733477341F344E343D344F3447348612A7
:10032800000006088D0086160800061100000D085A
:10033800860006150800003066002D30860006117C
:100348004708860000000615061008008D016400A5
:100358008C30620008308E008518BD29051DB02933
:10036800851103108D0C851CB72985158E0BB029B6
:1003780008000519B029051003148D0C051DC229A4
:1003880005148E0BB029080010308F0086108611D6
:100398000E30062086148615113006208F0BCA29C8
:1003A800080086140611000048088600061500009B
:1003B8000611000049088600061500000611000015
:1003C8004A0886000615000086100800AA210D08B4
:1003D800860006288617061FEF29861308000030B6
:1003E8006600AA210D0886000628FF306600060868
:1003F8008D0047220628C90DC90DCA0DC90DCA0DA1
:10040800C90DCA0D0F30C90508000430C800CA015B
:100418004808C900FF2149088C0006160000C701DA
:100428009F21D521FF306600EE2147109321FE3031
:100438000D020319232A4714CA01CB01080093218E
:100448000D08CA000D08C80093210D08CB000D083F
:10045800C9008C038C080319462A2030C807031CDE
:10046800392AC90A031C392ACA0AC908031D402A9D
:1004780020304802031C112A2030C802031C312AEC
:10048800C903312A080064008C30620008308E00ED
:10049800851C4C2A051D4C2A03108D0C03185D2A57
:1004A80005100519552A0514051D582A8E0B4C2AC6
:1004B800652A851185185E2A8515851C612A8E0B8B
:1004C8004C2A851C652A051D652A08009B308C006E
:1004D80064008C30620000008C0B6F2A080010301A
:1004E8008F000C3006200F3006208F0B752A08006D
:1004F80008308F00752A0D308F00752A86108611F6
:100508001108062086148615120806208F0B822AE9
:1005180008000630650034306600193085000A305E
:10052800860064008C3062000516061D032B861EAB
:10053800FF2AC801CA01AA210D08C900FF21C70165
:100548009F21D521FF306600EE21932188300D02CE
:100558000319B22A8D0147220616062808308C0096
:10056800932147228C0BB22A06160628AA210D08C9
:10057800C800AA210D08C90009224A088D0047228F
:100588004B088D004722471CCC2A06164710062820
:1005980093210D088C0047228C0A932147228C0B4B
:1005A800D12A06160628AA210D08C800AA210D0876
:1005B800C90009224A088D0047224B088D004722AE
:1005C800471CE92A06164710062893210D088C00B7
:1005D80047228C0A0C08CA07031CF32ACB0A1D30D1
:1005E8008C0093214722CA03031CFD2ACB0303185E
:1005F800DE2A8C0BF52A0519851C362B952A861EB2
:10060800062B952A8D010512061E0A2B08308E002E
:100618007C220619952A7322061D03100619031455
:100628008D0C8E0B0F2B73220619952A061E1C2B78
:1006380047227F22952AAA21A1300D0203199D2A5B
:10064800A2300D020319BA2A12300D020319F32938
:1006580010300D020319F92914300D020319EA2983
:10066800EE211F2B0512861ACF2B061E682B85013B
:10067800860106306500343066005123A723013017
:10068800460203194C2B0230460203194F2B412B0B
:1006980006087E23412BA723412B01306500640007
:1006A8000518532B6400051C562B1830C500C601CD
:1006B80001308023A7234608C500A723A53046029A
:1006C800031D512BA5307E2BAA2108308E00C8218E
:1006D80003108D0C0318742BC8218E0B6C2B772BF1
:1006E80073228E0B6C2BC8217F226A226A226A220F
:1006F8006A22952AC6000830C600051064000B302F
:100708008100051C852B4508C5000000C50B892BF9
:10071800C5000030C60C031C972B65000130C50BC3
:10072800922B65009E2B650001309A2B9B2BC50BE5
:10073800982B6500C60B872B4508C5000000C50B24
:10074800A22B640008000830C600051064000B30B6
:100758008100051CAD2B4508C5000030650001303F
:10076800C50BB32B6500B82BB92BBA2BC5010518DF
:10077800BB2BC50A45084502051CBD2BC60CC60B7C
:10078800BA2B0518C52B6400080000306600073036
:10079800C600C6018601AA210D0890008C00AA2176
:1007A8000D088F00AA210D089100AA210D089200BA
:1007B80013308400AA210D088000840A8C0BDE2BDC
:1007C800133084000F088D0008308E000D088F004C
:1007D80064008C3062000310800D031CF52B82220C
:1007E800F62B96208E0BEA2B840A900BE82B6A22B4
:0207F800952A40
:1042000000000000000000000000000000000000AE
:10421000000000000000000000000000000000009E
:10422000000000000000000000000000000000008E
:10423000000000000000000000000000000000007E
:10424000000000000000000000000000000000006E
:10425000000000000000000000000000000000005E
:10426000000000000000000000000000000000004E
:10427000000000000000000000000000000000003E
:084000007F007F007F007F00BC
:02400E00F53F7C
:02FFFE00840F6E
:00000001FF
